:020000040800F2
:10000000C0080020C900000805290008E9230008ED
:1000100000000000000000000000000000000000E0
:100020000000000000000000000000000929000896
:100030000000000000000000072900080B2900084C
:10004000DB00000800000000DB000008DB00000807
:10005000DB000008DB0000086D05000877050008DC
:10006000000000003D0500084D0500085D05000882
:1000700049020008DB000008DB0000080000000067
:10008000DB0000080000000000000000012A00085A
:1000900000000000DB000008DB000008DB000008B7
:1000A00000000000DB00000800000000ED31000847
:1000B0000448854600F0B6F8004800473133000890
:1000C000C046C046C0080020044880470448004796
:1000D000FEE7FEE7FEE7FEE7FEE7FEE7FF29000892
:1000E000B100000830B50B46014600202022012453
:1000F00009E00D46D5409D4205D31D469540491B5C
:100100002546954040191546521E002DF1DC30BDA4
:1001100070B500242546002801DA01244042002958
:1001200001DA01254942FFF7DDFFAC4200D0404231
:10013000002C00D0494270BDF0B51FB40646002027
:1001400082B005464024019100901BE001992246AF
:100150000F46304600F020F8049A059B801A99411A
:1001600010D310461946224600F04BF8361A8F413C
:100170000197224601200021009F00F042F8381824
:100180004D4100902046641E0028DFDC019B009852
:100190002946324607B0F0BD10B5202A04DB0846D8
:1001A000203AD040002110BD0B46D340D04020243F
:1001B000A21A91400843194610BD03460B439B0702
:1001C00003D009E008C9121F08C0042AFAD203E0CC
:1001D0000B780370401C491C521EF9D27047D2B2F2
:1001E00001E00270401C491EFBD270470022F6E776
:1001F00010B513460A4604461946FFF7F0FF20469D
:1002000010BD10B5202A04DB0146203A91400020A1
:1002100010BD914020239C1A0346E34019439040AF
:1002200010BD0000064C0125064E05E0E36807CC32
:100230002B430C3C98471034B442F7D3FFF73CFFF4
:10024000443700086437000810B5024800F063FA2C
:1002500010BD0000B802002070B504460068816837
:10026000490727D5816810254907002905DA8168E3
:10027000890702D481682943816000F05FFF064648
:1002800020688068400715D500F058FF801B0228C1
:100290000CD920688068400708D5A06B2843A0636C
:1002A000E06B01210843E063084670BD2068806868
:1002B0004007E9D4002070BD10B50246406A816B4A
:1002C000502319420AD1816B0122520211438163EA
:1002D0000168CA681205920F05D020E0006B016B1F
:1002E0001046884710BD827E002A18D10A6812077E
:1002F00015D58A6801235207002A09DB4A680C24B5
:10030000A2434A60816B1A0291431943816306E05C
:10031000816B202211438163C16B1943C16300F0DB
:10032000F7F910BD10B5406A816B4022114381631B
:10033000C16B04221143C16300F0ECF910BD10B58C
:10034000406A00F0E6F910BDF8B50446006881681F
:100350008907890F01292FD10168C90702D1C16816
:10036000090429D58168052211401025012601299B
:1003700016D1816802221143816021680320086040
:1003800000F0DCFE074620688068C00714D000F04B
:10039000D5FEC01B02280BD920688068C00707D093
:1003A000A06B2843A063E06B3043E0630120F8BDFD
:1003B00020688068C007EAD10020F8BDF8B504467F
:1003C00000200090206881688907890F012905D1E4
:1003D0000168C90736D1C168090433D481681A4A53
:1003E00010261140012500291FD181682943816011
:1003F000174816490068FFF775FE0090002802D0E4
:10040000401E0090FCD100F099FE0746206800686D
:10041000C043C00716D000F091FEC01B02280CD9C3
:1004200020680068C043C00707D0A06B3043A063BA
:10043000E06B2843E0630120F8BD20680068C043FA
:10044000C007E8D10020F8BD1700008040420F002F
:100450003000002010B5244C012023881A464100AA
:10046000615A994201D90B4602E0914200D20A46F4
:10047000401CC0B2FA28F2D3981A1C4C002802DDA6
:10048000E1894018E0812079411C217104282AD398
:100490000E200521205EFFF73BFE15494843154914
:1004A000FFF736FE1621615E00B248430A21FFF7CE
:1004B0002FFE01216156414308B2E0810C21615EAB
:1004C000411A0A31142900D9A081E078012802D00C
:1004D000002803D004E0A089208201E0A089608286
:1004E0000020E081207110BD3400002000000020B9
:1004F000E40C0000FF0F000041780278080210436E
:1005000040BA704770B4FF234A1E1C4692B20029BD
:100510000CD0084D084E0178401C59406B5C63407C
:10052000745C1146521E92B20029F4D11802204385
:1005300070BC70472C3500082C36000810B50248F6
:1005400000F03AFB10BD0000F802002010B5024890
:1005500000F032FB10BD00001804002010B5024866
:1005600000F02AFB10BD00005C04002010B508203C
:1005700000F016FD10BD10B5802000F011FD10BD7B
:1005800072B6FEE770B5044600F0D8FD1A4D064677
:10059000E868C0070DD0601C08D0002C04D000F023
:1005A000CDFD801BA04201D9032070BDE868C007C3
:1005B000F1D1E868800601D52020E860E868C0062F
:1005C00002D4E868400715D5E9680020CA060B493F
:1005D00004D5C86902221043C8611020EA68520796
:1005E00005D5CA6901231A43CA6104210843E8609A
:1005F000012070BD002070BD00200240A00400203A
:10060000F8B50025044620340095227D012A39D012
:1006100001262675026893685B0767D4384F4B68DC
:10062000BB424DD0936A0F78BE403343936201239F
:10063000C26A1B079A421FD0012A1DD0022A1BD072
:10064000032A19D0042A17D0052A15D0062A13D058
:10065000072A11D002688B6856697607760FB34275
:100660000AD05369DB08DB005361006842690B7AEA
:100670005B075B0F1A4342610868102804D01128F9
:1006800002D038E00220F8BD1E4B9A68102807D02F
:100690000120800502439A600868102803D02AE0F0
:1006A0000120C005F6E7194817490068FFF71AFD51
:1006B0000A21484300901ED0401E0090FCD11AE051
:1006C000906A0B789E40B04390620868102801D071
:1006D000112810D10B498A68102804D00120800508
:1006E00082438A6007E00120C005F9E7816B202280
:1006F000114381630125002020752846F8BD0000C4
:10070000011000000027014040420F00300000208F
:1007100070477047704770B5044600680168490724
:1007200002D54168490705D40168090730D54168F9
:1007300009072DD5A16BC90604D4A16B0122520271
:100740001143A163C1680C250905890F00291AD13D
:10075000A17E002917D10168090714D581680122FB
:100760004907002908DB4168A9434160A06B1102D9
:1007700088431043A06306E0A06B20210843A063D8
:10078000E06B1043E0632046FFF7C2FF206805607E
:100790002068016809060DD5406800060AD5A06BDF
:1007A000012109040843A063204600F0D9F821681C
:1007B0008020086020680168C90613D54168C90611
:1007C00010D5A16A1025012902D0C168C90707D038
:1007D000E16B02221143E16305602046FFF79AFFB7
:1007E0002068056070BD0000F8B5002504460028AB
:1007F00005D0A06B26462036002802D007E0012055
:10080000F8BD0020E0633075204600F0ABF8A06B27
:100810001022C006002870DB2068816849076CD46C
:10082000A16B1301994302231943A16381688907CE
:10083000890F012905D10168C9070FD1C1680904D1
:100840000CD4C16818239943A3681943C160206878
:100850000169636889008908194301612068C168DA
:100860003D4B1940C160207E8103607EC00301437F
:10087000A07E43031943A36A012B02D001231B036B
:1008800000E000231943E36819432369022B09D0D0
:10089000002319433379E67E5B0019430123012EBF
:1008A00002D00AE00423F4E7002827D0A06B20261A
:1008B0003043A063E06B1843E063E0690646FF3E07
:1008C000C23E02D0266A304301432068C6680E4308
:1008D000C6600126E06A3607B04213D0012811D065
:1008E00002280FD003280DD004280BD0052809D0EA
:1008F000062807D0072805D010E028E001200004D2
:100900000143DAE720684669F608F6004661206888
:100910004669A78D7F077F0F3E4346612068C06808
:100920000E4E3040884207D10020E063A06B800863
:100930008000401CA06308E0A06B022188431043A4
:10094000A063E06B1843E06301252846F8BDA06B67
:100950001043A063F8E700001902FEFFE7FF3F83A2
:100960007047000070B586B00024054600940194DD
:1009700002940394049400681E49884237D11E48AB
:100980008169421511438161816911400591426974
:10099000012149040A434261406908400590022050
:1009A00000900320019009206946C00600F004FB76
:1009B000134E12487460B46030608020F0604000D4
:1009C0003061800070612020F461B061304600F039
:1009D00045F9002801D0FFF7D3FD2E630022114610
:1009E0000C20756200F044FC0C2000F035FC06B0D1
:1009F00070BD0000002401400010024008000240C9
:100A0000F8020020F7B5044600680025806840071A
:100A10003ED426462036307D01280AD0012737757E
:100A2000607E012808D02046FFF7C8FC050003D0EF
:100A30002FE0022003B0F0BDA06B17490840FF2152
:100A400001310843A0630020E0633075216B134837
:100A50008862216B1248C862216B124808632168C2
:100A60001C20086020684168102211434160206802
:100A7000C1683943C1602168206B4031029B019AF3
:100A800000F020F92068816804221143816000E0B1
:100A90000225284603B0F0BDFEF1FFFFB9020008B1
:100AA0003F03000825030008F8B506460446203633
:100AB000307D012807D0012737752046FFF7CCFB92
:100AC000050002D02AE00220F8BD2068C16849086C
:100AD0004900C160206B014620304078022808D1CF
:100AE000084600F01FF8050003D0A06B4021084322
:100AF000A06320684168102291434160002D204688
:100B000002D0FFF721FC09E0FFF71EFC050005D12C
:100B1000A06BFF21013188433843A063002030756A
:100B20002846F8BD014620314A780023022A04D025
:100B3000042282630B700120704730B4026814688D
:100B40000E25AC43146002681468640864001460E5
:100B50000125046C2A46C06BA24042604D700B70A8
:100B600030BC0020704770B50024014620314A781F
:100B7000022A03D004218163012416E0026813686D
:100B80000E25AB431360026813685B085B001360BB
:100B90000125036C2A469A40C36B5A604D700022AF
:100BA0000A70416B002900D08847204670BD806BD9
:100BB0007047203040787047F0B4C16B0C68016812
:100BC0000B680426056C3246AA40224210D05A0710
:100BD0000ED50A68920602D40A68B2430A60016C14
:100BE0008E40C16B4E60C16A002935D1F0BC7047A0
:100BF0000227AF400246274001262032002F15D0A1
:100C00009F0713D50B689B0604D40B680A24A343E3
:100C10000B605670036C02219940C36B5960002130
:100C20001170816A002917D1F0BC70470827AF40C6
:100C30002742F9D01B07F7D50B680E24A3430B609E
:100C4000016C33468E40C16B4E608363537000214C
:100C50001170016B0029E7D0F0BC0847002801D1D2
:100C60000120704770B50446022025462035687083
:100C7000206802681049A3680A4061682669194320
:100C8000E3683343194363691943A3691943E3696B
:100C90001943114301600949206840181421FFF7E6
:100CA00021FA800020640648E0630020A06301214F
:100CB0006970287070BD00000FC0FFFFF8FFFDBF16
:100CC00000000240F0B40446944620342278002507
:100CD000012A0AD00127277066780022012E07D04A
:100CE000227002252846F0BC7047F0BC02207047F5
:100CF00002266670826302681468640864001460E7
:100D0000046C3E46A640C46B62466660046863603D
:100D10004368102B03680AD099600168CA60C16AF1
:100D2000002901680A6806D00E231A430AE09A6077
:100D30000268D160F3E70A231A430A6001680A686F
:100D400004239A430A600068016839430160C9E7D7
:100D5000F3B5054681B0012000902E48017E01299F
:100D60000DD00121017628682B4C2C4E40270128FC
:100D700008D02046FFF706FC002819D044E00220E6
:100D800003B0F0BD2046FFF7FDFB00283CD1214910
:100D9000C8613069042528433061306938433061C7
:100DA0002046FFF7EFFB00903069A84330612BE04D
:100DB00000210298C9430160A8686C68800200198C
:100DC000A04221D913490020C86130690227384365
:100DD0003061746130694021084330610E48FFF78B
:100DE000D1FB00903069B84330610098002802D0F0
:100DF0000298046008E0012080022418A86869684D
:100E000080024018A042DDD80249002008760098F0
:100E100003B0F0BDA004002050C300000020024039
:100E200003480169802211430161002070470000DE
:100E300000200240F0B51FB405461D480024017E85
:100E4000012907D0012606761A48FFF79BFB0028E8
:100E500003D027E0022005B0F0BD012D02D0022D05
:100E600000D00425002D1DD9134E019861000F18E4
:100E7000220103990298FFF78FF90D4A0021D161F1
:100E8000316901221143316138800A48FFF77AFB4A
:100E90003169490849003161002803D1641CE4B27A
:100EA000AC42E2D3024A0021117605B0F0BD000049
:100EB000A004002050C3000000200240064900208A
:100EC0000A69120607D5054A4A60054A4A60096957
:100ED000090600D501207047002002402301674524
:100EE000AB89EFCDF8B50927FF06012600242A4D6E
:100EF00080280DD008280AD12849022002F002FAE1
:100F00000821384600F006F901281BD0EC70F8BD26
:100F10004021384600F0FEF8012802D1A879401C93
:100F2000A8716879401CC0B268710528EFD9A8790A
:100F3000032801D36E7002E00020C04368706C711A
:100F4000AC71F8BDEE7010201221285E695E401A67
:100F5000032164280BDDE879401CC0B2E871032846
:100F600001D3AC702C72FA280CD9E9710AE0287A06
:100F7000401CC0B22872032801D3AE70EC71FA286D
:100F800000D929720C20285E4B21FF30C9002D307A
:100F90008842D6D8AC70F8BD00000020881300004D
:100FA00004494A69024204D010B54861FFF79AFF2C
:100FB00010BD7047000401400B680022002B72D066
:100FC000F8B401270B6897403B406DD00C79A4071B
:100FD000A40F012C01D0022C10D1856854000326E7
:100FE000A640B543CE68A6402E43866044680D797E
:100FF000BC43ED06ED0F9540254345600C79E44375
:10100000A40708D0C56854000326A640B5438E68DF
:10101000A6402E43C6600C79A407A40F022C0CD165
:10102000D408A40027183D6A5407E40E0F26A640F2
:10103000B5430E69A6402E433E6205685400032660
:10104000A640B5430E79B607B60FA6402E430660FC
:101050004C68A403A40F49D0284CA5690126354348
:10106000A561A469950834400094254CAD002F1962
:10107000BD689407240F0F26A640B5430926F6063F
:10108000B04201D1002611E01E4EB04201D101262E
:101090000CE01D4EB04201D1022607E01B4EB042CB
:1010A00003D1032602E028E020E00526A6402E43D7
:1010B000BE60174D2C684E689C43F60300D51C4358
:1010C0002C606C684E689C43B60300D51C436C6072
:1010D000AC684E689C43F60200D51C43AC60EC68DB
:1010E0004E689C43B60200D51C43EC600B68521C52
:1010F000D34000D065E7F8BC70477047001002404D
:10110000000001400004004800080048000C0048AE
:10111000000401400069084000D001207047426986
:1011200013460B401B0491430B4383617047002A15
:1011300001D081617047816270470000014880687A
:101140007047000024000020002801D101207047D2
:1011500070B5044621681648086021681548086083
:101160002068616841602168A0688860FFF7E6FF39
:1011700005462068C06840070ED0FFF7DFFF401B20
:10118000272805D92068C068400701D0032070BD1A
:101190002068C0684007F0D120680269E1688A428F
:1011A00001D0016101E004490160002070BD000030
:1011B000CCCC000055550000AAAA000000680249E6
:1011C0000160002070470000AAAA000010B5064880
:1011D0000168102211430160032000F007F800F0BD
:1011E00027F8002010BD00000020024070B5044622
:1011F0000D4D7D202978C000FEF774FF01460B4895
:101200000068FEF76FFF00F099FB002809D1042C5D
:1012100007D200222146401E00F02AF800206C6010
:1012200070BD012070BD00002400002030000020AF
:10123000084881B0816901221143816181691140AF
:101240000091C26901040A43C261C069084000906C
:1012500001B0704700100240002805DBC106C90E2E
:1012600001208840014908607047000000E100E06B
:101270008207D30EFF229A408907090E9940002861
:1012800008DB830809489B001818036893430B4345
:10129000036070470007000F0838830804489B006C
:1012A0001818C36993430B43C361704700E400E01F
:1012B00000ED00E0F8B504460068394EC0035AD589
:1012C000F0690025C00007D4F06931040843F061DB
:1012D000F06908400125009032480168C90515D41D
:1012E0000068FF21013108432E490860FFF726FFFF
:1012F00007462C480068C00508D4FFF71FFFC01B35
:10130000642825D827480068C005F6D5306A03212F
:101310000902084021D062680A4082421DD0306A2A
:10132000326A8843012109040A433262326A8A43DD
:1013300032623062C00710D0FFF700FF0746306A04
:1013400080070AD4FFF7FAFEC11B1748814201D972
:101350000320F8BD306A8007F4D5306A0321090202
:101360008843616808433062002D04D0F069012190
:1013700009078843F0612078C00705D0306BA16869
:1013800080088000084330632078800605D5306BE4
:1013900010218843E168084330630020F8BD000055
:1013A000001002400070004088130000002801D1A6
:1013B00001207047F8B504463E480D460068C00756
:1013C000C00FA8420AD23B48016849084900294396
:1013D00001600068C007C00FA84250D12068364E97
:1013E00081070CD5400704D570680721090208431E
:1013F00070607068F0218843A168084370602078AD
:10140000C0072CD0606801281BD0316802281CD08E
:10141000890734D571688908890001437160FFF735
:101420008DFE7168074662680C200140920091426F
:1014300015D0FFF783FEC11B2048814208D9032045
:10144000F8BD316889031AD5E4E7890117D5E1E7CA
:1014500070680C210840616889008842E9D115480C
:101460000168C907C90FA9420BD901684908490099
:10147000294301600068C007C00FA84201D00120C5
:10148000F8BD2078400706D5706807210902884317
:10149000E1680843706000F027F87168084A09069F
:1014A000090F515CC840074908600320FFF79EFE02
:1014B0000020F8BD00200240001002408813000008
:1014C0002C370008300000200448054900684968AE
:1014D000044A4905490F515CC8407047300000205C
:1014E000001002403C37000810B514A00FC888B0A7
:1014F0006C460FC415A00FC80FC4184A53680C20BF
:10150000194601401648042916D0082914D1990219
:10151000090F6C46645CD16A04AA0907090F525C82
:10152000D90305D500231946FEF706FE214601E042
:1015300020460C4901F0ACFE08B010BD02030405C2
:10154000060708090A0B0C0D0E0F10100102030408
:1015500005060708090A0B0C0D0E0F1000100240BB
:1015600000127A0000093D00002801D101207047D7
:10157000F8B504460078EE4DC00754D068680007FF
:10158000800F012807D068680007800F022809D162
:101590006868C00306D52868800344D560680028C1
:1015A00074D040E0606801280CD001218904002833
:1015B0000DD0052825D02A68881082432A60286823
:1015C00088430BE0286801210904084306E02868E5
:1015D00001221204904328602868884328606068CC
:1015E000002812D0FFF7AAFD0646286880031AD407
:1015F000FFF7A4FD801B642873D828688003F7D503
:1016000011E0286808432860DCE7FFF797FD0646ED
:101610002868800307D5FFF791FD801B642860D8F8
:1016200028688003F7D42078800741D568680007D0
:10163000800F07D068680007800F022809D168680A
:10164000C00306D42868800718D5E06801281DD19A
:1016500014E0E0680028286819D0012108432860B8
:10166000FFF76CFD06462868800707D4FFF766FD84
:10167000801B022835D828688007F7D52868F8210C
:1016800088432169C9000843286011E04CE1400803
:1016900040002860FFF752FD06462868800707D5FE
:1016A000FFF74CFD801B02281BD828688007F7D461
:1016B0002078000727D5E0690028686A12D0012148
:1016C00008436862FFF73AFD0646686A80071AD445
:1016D000FFF734FD801B022803D8686A8007F7D51E
:1016E00011E08BE0400840006862FFF727FD0646E6
:1016F000686A800707D5FFF721FD801B02287DD887
:10170000686A8007F7D4207804264007002866DA44
:10171000E8690027C00007D4E869B1060843E8611A
:10172000E86908400127009082480168C90515D47E
:101730000168801501437F480160FFF7FFFC0090BE
:101740007C480068C00509D4FFF7F8FC0099401AEE
:1017500064287DD877480068C005F5D5A0680128C1
:101760000AD0002801D005281ED0286A4008400071
:101770002862286AB04302E0286A012108432862EF
:10178000A068002814D0FFF7D9FC0090286A8007D1
:101790001ED4FFF7D3FC0099411A6748814257D8FD
:1017A000286A8007F5D513E0286A30432862E3E70A
:1017B000FFF7C4FC0090286A800709D5FFF7BEFC3C
:1017C0000099411A5C48814242D8286A8007F5D4C2
:1017D000002F04D0E869012109078843E8612078D7
:1017E000C0061BD56069012834D0401D686B4ED0FF
:1017F00030436863686B4008400000E028E068639D
:10180000FFF79CFC0646686B800707D5FFF796FC40
:10181000801B02281CD8686B8007F7D4206A002838
:1018200068D069680907890F022968D00126360641
:10183000022828682ED0B0432860FFF77FFC0446BA
:101840002868800172D5FFF779FC001B022852D965
:101850000320F8BD686B30436863686B012108435F
:101860006863FFF76BFC0646686B800707D4FFF7D9
:1018700065FC801B0228EBD8686B8007F7D5686B86
:10188000F8218843A169C90008436863C6E7B043EB
:101890006863F4E7B0432860FFF750FC0746286808
:1018A000800107D5FFF74AFCC01B0228D0D8286862
:1018B0008001F7D4E86AE16A000900010843E862A0
:1018C000616AA06A084369683D2212049143084393
:1018D0006860286830432860FFF730FC04462868B9
:1018E000800123D4FFF72AFC001B0228B0D8286807
:1018F0008001F7D51AE028688001A4D416E00128F9
:10190000A7D06868E96A01221204636A02409A4219
:101910000AD10907E26A090F914205D10F21890412
:101920000840A16A884201D00120F8BD0020F8BD1E
:101930000010024000700040881300000B4910B4F2
:10194000401E884202D910BC0120704708494861F6
:1019500008480722C3691B021B0A4C042343C361C6
:10196000002088610A6110BC70470000FFFFFF0083
:1019700000E000E004ED00E070477047002801D16E
:101980000120704770B5054604462035687F002861
:1019900003D12877204600F015F802206877211D32
:1019A000206801F035F801204034A071A877E8776D
:1019B00020706070A070E070207160716877002006
:1019C00070BD000008B50068094988420FD1094878
:1019D000C26981150A43C261C069002208400090B3
:1019E00001211320FFF744FC1320FFF735FC08BD4D
:1019F0000020004000100240014620314A7F012AA9
:101A000001D00120704702224A770168CB68012289
:101A10001343CB6000680849884202D007498842D6
:101A200004D181684907490F062902D00168114392
:101A30000160002070470000002C014000040040BD
:101A4000704770B50446006801690025C9438907DD
:101A5000002915DBC168C943890711D4E91E01615A
:101A600001202077206880698007204602D0FFF798
:101A7000E7FF04E000F096F8204600F04FF92577E4
:101A800020680169C943490717D4C168C943490798
:101A900013D40421C94301610220207720688069A2
:101AA0008005800F204602D0FFF7CAFF04E000F057
:101AB00079F8204600F032F9257720680169C9439A
:101AC000090716D4C168C943090712D40821C943BC
:101AD0000161042020772068C0698007204602D079
:101AE000FFF7AEFF04E000F05DF8204600F016F9C5
:101AF000257720680169C943C90617D4C168C9435D
:101B0000C90613D41021C943016108202077206839
:101B1000C0698005800F204602D0FFF791FF04E0E6
:101B200000F040F8204600F0F9F8257720680169B8
:101B3000C943C90708D1C168C943C90704D1891E6F
:101B40000161204600F05EF920680169C943090679
:101B500009D4C168C943090605D48021C94301617C
:101B60002046FFF709FF20680169C943490609D4E7
:101B7000C168C943490605D44021C94301612046D3
:101B800000F041F920680169C943890609D4C16898
:101B9000C943890605D42021C94301612046FFF7C6
:101BA000ECFE70BD70470000F8B5044600202646E4
:101BB00020360090307F0D4601280FD001200427E9
:101BC0003077002A0CD0042A1CD0082A2FD00C2AE7
:101BD0003FD00090002030770098F8BD0220F8BD7B
:101BE000206800F061FF206881690822114381614B
:101BF00020688169B9438161206881692A6911433C
:101C00008161E7E7206800F08DFF2068816901228B
:101C1000D202114381612068816952109143816130
:101C2000206881692A69120211438161D2E7206824
:101C300000F0B4FF2068C16908221143C161206827
:101C4000C169B943C1612068C1692A691143C16191
:101C5000C0E72068016A0122120391430162026A0F
:101C60004168C76973231B029F432B681B023B43D8
:101C700001277F03BA43AF683F031743124A9042DC
:101C800005D0124A904202D0114A904205D1012259
:101C9000920391436A69920111434160C36169688B
:101CA000016407622068C1690122D2021143C16147
:101CB0002068C16952109143C1612068C1692A69D5
:101CC00012021143C16185E7002C0140004401402C
:101CD00000480140002801D10120704770B5054639
:101CE00004462035687F002803D12877204600F07D
:101CF00014F802206877211D206800F089FE012079
:101D00004034A071A877E87720706070A070E07010
:101D1000207160716877002070BD704770470000C7
:101D200030B502460446002520324030002908D054
:101D3000042908D0082908D04378012B07D00120B6
:101D400030BD937FF9E7D37FF7E70378F5E7022308
:101D500000290ED004290ED008290ED04370002986
:101D60000DD0042910D0082914D00C2918D0012531
:101D70003DE09377F3E7D377F1E70370EFE720686F
:101D8000C2681A43C26010E02068C26804231A4384
:101D9000C2600AE02068C26808231A43C26004E0F7
:101DA0002068C26810231A43C2600122206800F034
:101DB0006DFE104A2068904205D00F49884202D03B
:101DC0000E49884204D1416C0123DB03194341646D
:101DD00020680123904202D00949884204D18168D9
:101DE0004907490F062902D00168194301602846B6
:101DF00030BD0000002C014000440140004801407B
:101E000000040040704770477047F8B5816F044682
:101E1000C66F006882682546120610278035002AA2
:101E200026DA212924D1EFF31081012282F31088D0
:101E3000826880239A43826081F31088E06E0028D4
:101E400008D0FEF76FFE002804D0E06EFEF7AFFE6C
:101E500020282FD0EFF31081012080F31088206814
:101E60000268C0239A43026081F310882020A06793
:101E70002068816849061BD5222E19D1EFF3108105
:101E8000012282F31088826840239A43826081F3A2
:101E90001088206F002808D0FEF744FE002804D0E8
:101EA000206FFEF784FE202804D0204601F008F8B9
:101EB0000020F8BD2F600320F8BD7047F8B5026818
:101EC0000446D069116896689F4B05461D40202343
:101ED000002D76D0F7079D4DFF0FBC460D402F43D8
:101EE0006ED02546C7078035002F06D0CF0504D514
:101EF000012717622A683A432A60820708D5F20749
:101F000006D0276802223A622A6804273A432A60E8
:101F1000420708D5F20706D02668042232622A68F2
:101F2000022632432A6002070AD50A461A4066464C
:101F3000324305D02668082232622E6816432E608E
:101F4000020508D54A0106D501222668D20232626E
:101F50002A681A432A602A68002A2FD0800606D5EC
:101F6000880604D5616E002901D02046884728687C
:101F700021688968490602D4282108422DD02046CC
:101F800000F09EFF20688168490622D5EFF310819A
:101F9000012282F31088836840229343836081F397
:101FA0001088206F002814D069494163206FFEF724
:101FB000DAFD002802D0206F416B8847F8BD00E0B1
:101FC00011E085060FD58D060DD5616E00297CD1F7
:101FD000F8BD2046FFF771FFF8BD2046FFF76DFF03
:101FE00000202860F8BD256E012D6FD1C5066DD586
:101FF000CD066BD5102717622068816825464906F3
:102000004035002948DA226F116849680904090C33
:10201000E8D02E8B8E42E5D969839169202933D08F
:10202000EFF31081012282F3108802683E01B2436F
:10203000026081F31088EFF31081012080F3108893
:102040002068826852085200826081F31088EFF3A2
:102050001081012080F31088206886684022964312
:10206000866081F31088E36700202066EFF310811B
:10207000012080F3108820680368BB43036081F36C
:102080001088206FFEF74EFD288B698B401A81B2B5
:102090002046FFF7B9FEF8BD298B6A8B891A6A8B37
:1020A00089B2002AF7D00029F5D0EFF3108201257C
:1020B00085F310880568FF262136B543056082F355
:1020C0001088EFF31082012001E023E01BE080F391
:1020D0001088206885686D086D00856082F310881F
:1020E000E36700202066EFF310826066012080F332
:1020F000108820680368BB43036082F31088204681
:10210000FFF782FEF8BD050607D50D0605D5A16EC1
:102110000029F7D020468847F8BD4006FCD5480680
:10212000FAD52046EFF31081012484F31088146857
:102130004025AC43146081F31088836700218166D9
:1021400000F050F9F8BD00000F0800002001000465
:10215000492D0008002801D10120704710B5044620
:10216000806F002805D1002174200155204600F021
:1021700027F82420A0672068016849084900016009
:10218000204600F0CDFE012818D0606A002802D059
:10219000204600F041FD206841680122D2029143AF
:1021A000416020688168082291438160206801684D
:1021B000012211430160204600F094FD10BD000093
:1021C000F0B587B00024054600940194029403946E
:1021D00004940068314988425DD131488269012107
:1021E00089030A43826182690A4005924269C900F3
:1021F0000A43426140690840059003204002009074
:1022000002200190032003900120049009206946D8
:10221000C006FEF7D1FE244E80277460B46034619E
:102220007461F7601F48B46130608014F06130461B
:10223000FEF714FD002801D0FEF7A2F92E677562A3
:102240001B4E1A483060B46034617461F76010202E
:10225000B46170600002F0613046FEF7FFFC0028B8
:1022600001D0FEF78DF91348016842151143016052
:10227000EE66002211461B207562FEF7F9FF1B2057
:10228000FEF7EAFF0C4B1868026810210A4302604F
:1022900019685020086207B0F0BD00000038014006
:1022A00000100240300002401804002044000240A8
:1022B0005C040020000001409403002070B5C36F4F
:1022C000202B2BD100290BD0002A09D001248368B0
:1022D0002403A34206D10369002B03D1CB0701D00D
:1022E000012070BD034660331C7D012C16D00124F3
:1022F0001C750023036603685C6824020BD5EFF3AA
:102300001084012585F310881D680126B606354323
:102310001D6084F3108800F093FE70BD022070BD34
:1023200070477047F8B50446806F202852D10029C5
:102330000BD0002A09D00123A0681B03984206D1C4
:102340002069002803D1C80701D00120F8BD254627
:102350006035287D01283DD0012028752046403079
:10236000E1640282428200272646803637602120BF
:10237000A067E06E00281BD017498162E16E174804
:10238000C862E16E16480863E06E13464763206832
:10239000E16C283084466246E06EFEF793FC00282C
:1023A00006D0102030602F752020A0670120F8BDD6
:1023B0002168402008622F75EFF31081012080F31F
:1023C00010882068826880231A43826081F3108815
:1023D0000020F8BD0220F8BD6D2E0008B72E0008C1
:1023E0005D2D000870477047FEE70000F0B54B4CCC
:1023F00085B0A01CFEF780F80746201DFEF77CF88C
:10240000064606212046FEF77DF8050AC4B2012FD4
:1024100002D0FF2F22D03CE0022E5DD13F488179CF
:10242000A94259D1C179A14256D13D4C01782170C0
:102430004078607004203B49A07088890212E270E5
:102440002071885701126171A07107212046FEF7A3
:1024500059F8010AE17120720B203BE0012E3BD1BB
:102460002E488179A94237D1C079A04234D12EA01B
:102470000FC80191039300902949029200206B46F6
:102480001A5C0A54401CC0B21028F9D3112000F085
:10249000F5FF0221022F21D0032F1DD1012E1BD1C8
:1024A0001E488279AA4217D1C279A24214D11C4C8B
:1024B00002782270407860701A48A170C08A0112B8
:1024C000E170207105212046FEF71CF8010A6171B8
:1024D000A071092000F0D2FF05B0F0BD012EFBD1A4
:1024E0000E488279AA42F7D1C279A242F4D10C4CAB
:1024F00002782270407860700A48A170808A010AD0
:10250000E170207105212046FDF7FCFF010A617191
:10251000A071092000F0B2FF05B0F0BD4802002014
:1025200028020020000000204443452D3233303281
:102530002D56345F48414C00F8B5454EB188B01C6B
:1025400049BA0CB2FDF7D8FF054606213046FDF723
:10255000D9FF01463F4F0020325C3A54401CC0B2C4
:102560000628F9D30A0ABA71C9B23B48F9710F2D8E
:1025700004D0022D2AD0032D3FD064E0B3799A42D3
:1025800061D1F27991425ED1611EF6290DD8448164
:10259000012080F3108800F091FF002853D180F3D0
:1025A0001088307800280DD14DE0FF203871787107
:1025B00006212748FDF7A6FF010AB971F8713078A6
:1025C000002840D00A2000F059FF3CE0B3799A423D
:1025D00039D1F279914236D1204A611E914232D8E6
:1025E000A1B281821E4800684163012080F31088F7
:1025F00000F064FF002820D025E0B3799A4222D170
:10260000F27991421FD11749174A611891421AD89D
:1026100022460A214A430C210546415E1046FDF739
:1026200077FDE882012C01D10A20E882012080F3A5
:10263000108800F043FF002805D1002080F31088A7
:102640000A2000F01BFF20210148FDF7CFFDF8BD57
:10265000480200202802002000000020E7030000BC
:102660004C030020E40C0000C819000010B584B031
:102670000021184800910191154A02910260816081
:102680000124520504614260C16004224261017666
:1026900041768476FF22C176C232C2610E4A01625F
:1026A00011718462FEF7A0F8002801D0FDF768FFE1
:1026B000012000030190072002900094694605481C
:1026C000FDF79EFF002801D0FDF75AFF04B010BDB2
:1026D00000240140B8020020D802002008B51048AC
:1026E000416901221143416140690121104000907C
:1026F00000220920FEF7BCFD0920FEF7ADFD0022F7
:1027000001210A20FEF7B4FD0A20FEF7A5FD0022F4
:1027100001210B20FEF7ACFD0B20FEF79DFD08BD4F
:102720000010024030B587B0002430480094019476
:102730000294039404944269012189050A43426189
:1027400042690A400592426949110A43426142695D
:102750000A400592426949000A43426140690925DD
:102760000840ED060590012210212846FEF7DFFC07
:10277000002220212846FEF7DAFC082000903120B4
:1027800000040190694602942846FEF715FC0121D9
:102790003020019103910090029469462846FEF78B
:1027A0000BFC402000900194694602942846FEF7F5
:1027B00003FC8020009011200004019069460294DF
:1027C0002846FEF7F9FB002202210620FEF750FD05
:1027D0000620FEF741FD002211460720FEF748FDC6
:1027E0000720FEF739FD07B030BD000000100240A1
:1027F00010B5094807490160062141600749C160D9
:10280000272109018160FEF79FFC002801D0FDF718
:10281000B7FE10BD003000403C030020FF0F000059
:1028200070B58EB0002400940194244D029403945A
:1028300004940594204E06942E600120AC606860DC
:102840002C611F48AC61E8602846FFF797F8002824
:1028500001D0FDF795FE1948FFF73CFA002801D09A
:10286000FDF78EFE60200090FF202D300190029435
:102870000022694604941148FFF796F9002801D018
:10288000FDF77EFE0794089409940A940B94286837
:10289000B0420FD10B484269012189040A434261C9
:1028A000406908400C9002200790089007A906484C
:1028B000FEF782FB0EB070BD002000404C030020EC
:1028C000E7030000001002400004004810B50C4867
:1028D0000A4901604B21C901416000218160C1604A
:1028E00001618161C1610C22016242614162FFF7B5
:1028F00031FC002801D0FDF743FE10BD0038014037
:1029000094030020FEE77047704700B500F002F81E
:1029100000BD000030B4194B58680124002804D0D1
:102920005868401E586000D11C70154D00210C20C5
:10293000484340194268002A09D04268521E42604A
:1029400005D144700278012A01D182684260491C95
:10295000C9B20429EBD39868401C98609868094A6A
:102960000021904200D199605878401CC0B2587044
:102970000A2800D3597030BC7047000018000020AE
:1029800088020020FFFFFF7F70B594B000240594FB
:1029900004940F94092002250E9400901394E803E8
:1029A00002940394069409900B940C940D940126C0
:1029B00000011094119412940A90019607960895BC
:1029C0006846FEF7D1FD002801D072B6FEE7072069
:1029D0000C900E9401210D950F940CA8FEF7E6FCC7
:1029E000002801D072B6FEE710A810961294FEF7E8
:1029F00061FC002801D072B6FEE714B070BD7047CC
:102A000010B50248FFF71DF810BD00004C03002070
:102A100070B40268184C194EA04201D0B04204D1E3
:102A2000134670254A68AB431A43154B154DA04217
:102A300008D0B04206D0144EB04203D0984201D024
:102A4000A84204D103263602B243CE683243802620
:102A5000B2434E69324302608A68C2620A68826287
:102A6000A04203D0984201D0A84201D10969016374
:102A70000121416170BC7047002C014000040040FE
:102A800000440140004801400020004010B4C90645
:102A9000C90E0123046A8B409C430462036A8A4086
:102AA0001343036210BC7047F0B4026A520852002C
:102AB0000262056A436882697024A24392080C6826
:102AC00092001443022295438A68134E2A43134FFF
:102AD000B04204D0B84202D0114DA84206D1082518
:102AE000AA43CD681543042295432A46B04204D038
:102AF000B84202D00A4DA84206D103252D02AB43AD
:102B00004D691D438B692B43436084614968416370
:102B10000262F0BC70470000002C014000440140FC
:102B200000480140F0B4026A10239A430262046A2A
:102B30004368826973252D02AA430D68144E2D0245
:102B40001543202294438A6812012243B04207D1E0
:102B50001446CA688027BC43120122434024A24382
:102B6000B04205D00B4CA04202D00B4CA04208D181
:102B70000324A402A3434C69A4001C438B699B005B
:102B8000234343608561496881630262F0BC7047FA
:102B9000002C01400044014000480140F0B4026AAA
:102BA000FF2301339A430262046A4368C2697025B5
:102BB000AA4392080D6892001543012252029443E1
:102BC0008A68124E12022243B04207D11446CA68E4
:102BD000C714BC43120222430415A243B04205D0DD
:102BE0000B4CA04202D00B4CA04208D1032424037A
:102BF000A3434C6924011C438B691B01234343609D
:102C0000C5614968C1630262F0BC7047002C014095
:102C1000004401400048014010B4818CC90707D02E
:102C200001684A6801235B049A43836A1A434A6035
:102C3000818C890707D501684A6801231B049A43E0
:102C4000C36A1A434A60818C490707D501684A68FC
:102C500001239B049A43036B1A434A60818C090742
:102C600007D501684A680123DB039A43436B1A4383
:102C70004A60818CC90607D501688A6801231B0355
:102C80009A43836B1A438A60818C890607D5016851
:102C90008A6801235B039A43C36B1A438A60818C61
:102CA000490612D501684B6801221205046C934352
:102CB00023434B60016C914207D101684A680323AA
:102CC0005B059A43436C1A434A60818C090607D519
:102CD00001684A680123DB04806C9A4302434A601E
:102CE00010BC7047F8B50446002580300560FEF73B
:102CF00025FA074620680068124E000709D5012111
:102D00003B46002249052046009600F0F3F90028D2
:102D10000DD12068006840070BD501213B460022F9
:102D200089052046009600F0E5F9002801D003202F
:102D3000F8BD2020A067E067256660342575002077
:102D4000F8BD0000FFFFFF0110B5406A00220146F8
:102D500040314A834A82FFF7B0F810BD70B5446A2B
:102D6000A06FE26F2168896800230906002911DA43
:102D700021280FD152200353EFF31081012080F35B
:102D8000108820680568C026B543056081F3108867
:102D90002020A06720688068400606D5222A04D13A
:102DA0005A200353204600F08BF8204680300168FB
:102DB0001022114301602046FFF77FF870BD10B567
:102DC00001468969406A202937D000225A210A52D7
:102DD000EFF31082012181F3108801680B68FF2452
:102DE0000134A3430B6082F31088EFF310820121BA
:102DF00081F3108801688B685B085B008B6082F34D
:102E00001088EFF31082012181F3108801688B682C
:102E10004024A3438B6082F310882021C167016E98
:102E200001290AD1EFF3108281F3108801680B6841
:102E30001024A3430B6082F31088016E012902D095
:102E4000FFF76EFA10BD5821095AFEF7DDFF10BDDD
:102E500010B5406A016E012902D0FFF762FA10BD79
:102E60005821095A4908FEF7CFFF10BD10B5014699
:102E70008969406A20291BD0002252210A52EFF3AF
:102E80001082012181F3108801688B688024A3439C
:102E90008B6082F31088EFF31081012282F3108897
:102EA0000068026840231A43026081F3108810BD55
:102EB000FFF798FA10BD10B5406AFFF794FA10BDFD
:102EC00010B4EFF31082012181F3108801680B68C0
:102ED000FF242134A3430B6082F31088EFF31082A8
:102EE000012181F3108801688B685B085B008B60AF
:102EF00082F31088016E01290AD1EFF3108281F369
:102F0000108801680B681024A3430B6082F31088BB
:102F10002021C16700210166416610BC7047000096
:102F200070B5044681680069E26901436069002563
:102F300010430143206802683C4B1A400A43026078
:102F400020684168032212039143E2681143416003
:102F5000216AA0690143206882680B231B029A43FF
:102F60000A4382603248006B8007800F06D0012838
:102F700016D0022816D0032810D010200122E369B1
:102F8000D2032C492C4E93422AD100280CD002287F
:102F90000DD004280DD008283ED10EE00220EDE728
:102FA0000420EBE70820E9E7FEF78EFA03E00A4683
:102FB00003E0FEF799FA020032D0616850004A0837
:102FC0008018FDF78FF880B201461039B14223D83E
:102FD0001A4901400007420F20680A43C2601FE0FF
:102FE000002806D0022807D0042807D0082813D1CB
:102FF00008E0FEF769FA03E00A4603E0FEF774FA18
:1030000002000DD0616848088018FDF76BF880B2A7
:1030100001461039B14201D9012501E02168C8609B
:1030200000206066A066284670BD0000F369FFFFBF
:103030000010024000127A00EFFF0000F0FF0000D5
:10304000F8B50446416540300027264602838036A5
:1030500037602220E0672546206F603500281BD0AE
:1030600021498162216F2148C862216F204808638D
:10307000206F13464763606D2168844662462431A1
:10308000206FFDF71FFE002806D0102030602F753E
:103090002020E0670120F8BD2F75EFF3108101209B
:1030A00080F3108820680268FF2301331A4302600E
:1030B00081F31088EFF31081012080F310882068DD
:1030C000836801221343836081F31088EFF310813A
:1030D00082F310882068826840231A43826081F35B
:1030E00010880020F8BD0000BF2D0008512E0008F8
:1030F0005D2D0008FFB50446006881B00E460A9DAC
:10310000C1691746304688433FD00020B84268D195
:10311000204660300090681C5BD0FEF70FF80499E1
:10312000401AA84233D8002D31D0206801684907E1
:103130004FD5C069C04300054BD401202168C002AF
:103140000862EFF31081012080F310882068026884
:10315000FF23A1339A43026081F31088EFF31081BB
:10316000012080F310882068826852085200826033
:1031700081F310882020A067E067803420600099E8
:1031800000200875032005B0F0BD0120BEE7EFF375
:103190001081012080F3108820680268FF23A1338A
:1031A0009A43026081F31088EFF31081012080F3CD
:1031B00010882068826852085200826081F310886B
:1031C0002020A067E067009900200875032005B063
:1031D000F0BD2068C1693046884305D00020B84260
:1031E00099D0002005B0F0BD0120F8E710B51148D6
:1031F000FEF764FE0F480068C169C943C90618D4C8
:10320000102101620B48FEF700FE0B4801780029EF
:103210000AD10A49096849682022511ACAB20270C3
:1032200007490848FCF7C9FF202205490148FFF774
:1032300045F810BD94030020000000201804002071
:10324000680200204802002010B50F480F4C027899
:1032500041786389204600789A4201D1082802D03B
:10326000002A08D00DE0032902D0062909D106E082
:10327000FFF7BCF805E0082803D1062901D1FFF7C4
:103280005BF90020207010BD4802002000000020E3
:10329000F0B4040C8BB2264682B25E430D0C10468D
:1032A000370C5843360480190021794116466E4385
:1032B000370C36048019794126466E438919F0BCD3
:1032C000704702E008C8121F08C1002AFAD17047EF
:1032D0007047002001E001C1121F002AFBD1704796
:1032E000042806D20C214843054940184178012999
:1032F00001D000207047002141700120704700007C
:1033000088020020042800D3FEE7012282F31088FF
:103310000C22064B5043C21851609160002151703D
:1033200001221A5481F3108870470000880200209F
:10333000FDF74CFFFFF728FBFFF7F4F9FFF7CEF995
:10334000FFF794F9FFF7C2FAFFF752FAFFF768FAAE
:103350003C493D4A08883D4B1080002801D09842E6
:1033600001D1012010804888394A0028108001D0FE
:10337000984202D17D20C0001080364A80B2126887
:1033800050630420085E34490028088001D0401CA6
:1033900001D10A2008803148FDF710FF2D48FEF7C3
:1033A0002BFB00212B48FEF7BBFC2D48FEF72DFD23
:1033B00020222C492A48FEF781FFFA222A492B486D
:1033C000FDF720FB092000222021C006FDF7AFFEFB
:1033D00032210020FFF796FFFF21F5310120FFF792
:1033E00091FF23490220FFF78DFF0225214E224C39
:1033F00000270020FFF774FF002809D01B48FDF7C5
:1034000053FBFDF727F8FA2217491848FDF7FAFA97
:103410000120FFF765FF002807D01048FDF7CEFE1A
:1034200009201021C006FDF77AFE0220FFF758FFA1
:10343000002800D0357020780028DAD0FFF704FF8C
:103440002770D6E7003C00080A000020FFFF0000BC
:10345000140000204C030020160000203C03002034
:10346000940300206802002034000020B8020020ED
:1034700088130000020000200000002070B509241D
:103480000546E406012220212046FDF750FE2A468B
:1034900007490848FEF746FF0748FDF78AFB012861
:1034A000FAD1002220212046FDF741FE70BD000028
:1034B00028020020940300205C04002010B586B090
:1034C0000020009001900290164C0120039404907B
:1034D000FDF7F4FC05A902A8FDF73AFC002802D08C
:1034E000012006B010BD104A694650890870000AD4
:1034F0004870908A8870000AC870D08A08710012DB
:10350000487121460320019B009AFDF793FC002897
:1035100002D0032006B010BDFDF782FC002006B0EB
:1035200010BD0000003C00080000002000C18140E8
:1035300001C0804101C0804100C1814001C0804183
:1035400000C1814000C1814001C0804101C0804173
:1035500000C1814000C1814001C0804100C1814063
:1035600001C0804101C0804100C1814001C0804153
:1035700000C1814000C1814001C0804100C1814043
:1035800001C0804101C0804100C1814000C1814033
:1035900001C0804101C0804100C1814001C0804123
:1035A00000C1814000C1814001C0804101C0804113
:1035B00000C1814000C1814001C0804100C1814003
:1035C00001C0804101C0804100C1814000C18140F3
:1035D00001C0804101C0804100C1814001C08041E3
:1035E00000C1814000C1814001C0804100C18140D3
:1035F00001C0804101C0804100C1814001C08041C3
:1036000000C1814000C1814001C0804101C08041B2
:1036100000C1814000C1814001C0804100C18140A2
:1036200001C0804101C0804100C1814000C0C10192
:10363000C30302C2C60607C705C5C404CC0C0DCD22
:103640000FCFCE0E0ACACB0BC90908C8D81819D992
:103650001BDBDA1A1EDEDF1FDD1D1CDC14D4D515C2
:10366000D71716D6D21213D311D1D010F03031F1B2
:1036700033F3F23236F6F737F53534F43CFCFD3DE2
:10368000FF3F3EFEFA3A3BFB39F9F83828E8E929D2
:10369000EB2B2AEAEE2E2FEF2DEDEC2CE42425E582
:1036A00027E7E62622E2E323E12120E0A06061A1F2
:1036B00063A3A26266A6A767A56564A46CACAD6DA2
:1036C000AF6F6EAEAA6A6BAB69A9A86878B8B97912
:1036D000BB7B7ABABE7E7FBF7DBDBC7CB47475B542
:1036E00077B7B67672B2B373B17170B05090915132
:1036F0009353529296565797559594549C5C5D9D62
:103700005F9F9E5E5A9A9B5B995958988848498951
:103710004B8B8A4A4E8E8F4F8D4D4C8C4484854501
:1037200087474686824243834181804000000000F3
:103730000000000001020304060708090000000061
:103740000102030464370008000000203400000078
:10375000C232000898370008340000208C080000AE
:10376000D23200080001010000000000000000004B
:103770000000000000000000000000000000000049
:103780000000000000000000010000000400000034
:083790000000000000127A00A5
:04000005080000B13E
:00000001FF
